:1000000085C200009FC200009DC200009BC200008C
:1000100099C2000097C2000095C2000093C2000080
:1000200091C200008FC200008DC200008BC2000090
:1000300089C2000087C2000085C2000083C20000A0
:1000400081C200007FC200007DC200007BC20000B0
:1000500079C20000D9C3000075C2000073C200005D
:1000600071C200006FC200006DC200006BC20000D0
:1000700069C2000067C2000065C2000063C20000E0
:1000800061C200005FC200005DC200005BC20000F0
:1000900059C2000057C2000055C2000053C2000000
:1000A00051C200004FC200004DC200004BC2000010
:1000B00049C2000047C2000045C2000043C2000020
:1000C00041C200003FC200003DC200003BC2000030
:1000D00039C2000037C2000035C2000033C2000040
:1000E00031C20000A0A1A1A01B09A51CA010A0A0C6
:1000F000201A0111B12C0D0E02160318A00B0A08CC
:1001000007060413A009151914120517A0A6A40DBB
:100110000A0F0CA0A01D1BA0A0C0BFBE00BDBCBB91
:10012000BAB9B8B7A8A9AAAB00C1ADACA0A1A1A0AB
:100130001B09A55C7F503B2F205A4151A02C4D4EEE
:1001400042564358A04B4A4847464453A049555944
:1001500054524557A0A6A40D0A4F4C2E7E5D5B2D30
:100160003A3039384037363534333231A8A9AAAB62
:1001700000C1ADACA0A1A1A01B09A57C7F502B3F65
:10018000205A4151B23C4D4E42564358A04B4A482A
:1001900047464453A049555954524557A0A6A40D6B
:1001A0000A4F4C3E7E7D7B3D2A302928602726253C
:1001B00024232221A8A9AAAB00C1ADACA0A1A1A073
:1001C0001B09A55C7F703B2F207A6171A02C6D6E9E
:1001D00062766378A06B6A6867666473A0697579F4
:1001E00074726577A0A6A40D0A6F6C2E7E5D5B2DE0
:1001F0003A3039384037363534333231A8A9AAABD2
:1002000000C1ADACA4A1A1A0A01BA515A010A05C2D
:10021000201A0111A05B0D0E02160318A00B0A088C
:1002200007060413A009151914120517A0A0A00DA4
:10023000A60F0C5DA0A0B15FA0C07D7B7F605EBB00
:10024000BAB97E7CA8A9AAAB00C1ADACA4A1A1A0FB
:10025000A01BA515A0503B2F205A4151A02C4D4E5C
:1002600042564358A04B4A4847464453A049555923
:1002700054524557A0A0A00DA64F4C2EA0A0A02DD3
:100280003A3039380837363534333231A8A9AAAB79
:1002900000C1ADACA4A1A1A0A01BA515A0402B3FFF
:1002A000205A4151A03C4D5E42564358A04B4A480B
:1002B00047464453A049555954524557A0A0A00D54
:1002C000A64F4C3EA0A0B23D2AA0292808272625EB
:1002D00024232221A8A9AAAB00C1ADACA4A1A1A04E
:1002E000A01BA515A0502B3F205A4151A03C4D4EBC
:1002F00042564358A04B4A4847464453A049555993
:1003000054524557A0A0A00D404F4C3EA0A0B23D76
:100310002A4029280827262524232221A8A9AAAB78
:1003200000C1ADACA4A1A1A0A01BA5157F703B2F5F
:10033000207A6171A02C6D6E62766378A06B6A681A
:1003400067666473A069757974726577A0A0A00D63
:100350005E6F6C2EA0A0A02D3A30393808373635A4
:1003600034333231A8A9AAAB00C1ADACA5A20113A8
:10037000040607080A0B0C0B0A7FB1A5A4A11A18E2
:100380000316020E0D0C0E0FA180A0A01B0102038C
:10039000040506070809000D1E1B1C1DB2091117D4
:1003A0000512141915090F10000D0A8CA8A9AAAB83
:1003B00000C1ADACB3978120939A8E8B2D372A382C
:1003C0002F39A0A0343135323633A0A0302E2BA0E7
:1003D000A0A0A0A0A5A24153444647484A4B4C3B8D
:1003E0003A5FA6A5A4A15A584356424E4D3C3E3F03
:1003F000A180A0A01B212223242526272829203DD7
:100400007E5B5C5DB20951574552545955494F5076
:10041000600D0A8CA8A9AAAB00C1ADACB39781202E
:10042000939A8E8B2D372A382F39A0A0343135324C
:100430003633A0A0302E2BA0A0A0A0A0A5A241538F
:10044000444647484A4B4C3B3A7FA6A5A4A15A587C
:100450004356424E4D2C2E2FA180A0A01B3132338B
:10046000343536373839302D5E5B5C5DB209515713
:100470004552545955494F50400D0A8CA8A9AAAB72
:1004800000C1ADACB3978120939A8E8B2D372A385B
:100490002F39A0A0343135323633A0A0302E2BA016
:1004A000A0A0A0A0A5A26173646667686A6B6C3B9C
:1004B0003A7FA6A5A4A17A786376626E6D2C2E2F62
:1004C000A180A0A01B313233343536373839302D76
:1004D0005E5B5C5DB20971776572747975696F7086
:1004E000400D0A8CA8A9AAAB00C1ADACB39781207E
:1004F000939A8E8B2D372A382F39A0A0343135327C
:100500003633A0A0302E2BA0A0A0A0A011241FBE87
:10051000CFEFD1E2DEBFCDBF13E0A0E0B2E0EAEA68
:10052000F9E102C005900D92AA30B107D9F724E095
:10053000AAE0B3E001C01D92A03AB207E1F7FBD6F2
:100540000C94A50C5DCD805A813208F037C0E82F9D
:10055000F0E0E955F34F12C7CEC3CFC3D2C3D6C321
:10056000E1C3E9C47EC385C38CC393C3B0C1CBC40C
:1005700087E06CC588E06AC589E068C581E066C52A
:1005800082E064C583E062C584E060C585E05EC545
:1005900086E05CC584E0D2C285E0D0C286E0CEC2EF
:1005A00087E0CCC288E0CAC289E0C8C28AE0C6C27D
:1005B0008BE0C4C28CE0C2C28DE0C0C20895815AF3
:1005C0008D3070F4E82FF0E0E853F34FD7C6AEC398
:1005D000AFC3C9C442C349C350C357C37BC17FC45F
:1005E0000895682F80910D0345C2CF93C82F813A9B
:1005F00018F0A9DFCF910895F4DF80910E038C17D6
:10060000C9F3C0930E0362D4F5CFCF93C82F8A30BD
:1006100041F06C2F80910C032DD28C2F90E0CF9164
:1006200008958DE0F2DFF5CFCF9380910C0355D282
:10063000C82F803A41F080910A0390910B035CD15E
:100640008C2FCF91089580910D0347D2C82FF8CFFA
:1006500090E090930B0380930A030895CF93DF9368
:10066000C82FD62F68D3482F6D2F8C2F16D3DF912C
:10067000CF9108956F927F928F929F92AF92BF9287
:10068000CF92DF92EF92FF920F931F93CF93DF935E
:1006900081E063D2A82EB92E83E050D200E00F2E65
:1006A000FAE07F2EF02D88248394912C0F2EF0EA0F
:1006B0006F2EF02D5AC08C2F90E0F701E80FF91F34
:1006C00020813FEF320F2130D1F03083D69516953F
:1006D000CF5F94D2C81708F047C0D0FDECCF10FF11
:1006E000F5CF6C2F802FBADF90910E038913EECFD8
:1006F00047D4882359F380910E0377DFE7CFF701C2
:10070000E80FF91F708210FF12C0F601E157FC4F8D
:1007100094010C2E02C0220F331F0A94E2F780814D
:10072000822B80836C2F802F99DF5FDFCFCFF60184
:10073000E157FC4F94010C2E02C0220F331F0A9484
:10074000E2F7C90180959081892380836C2F802FE7
:1007500085DF813A38F490910E038913B7CF609208
:100760000E03B4CF2CDFB2CF0F5F3DD20817C0F419
:10077000802FF5010995182FC02ED12CF601E157D5
:10078000FC4FD081D827C0E0C601880F991F880F81
:10079000991F880F991F9C01215F3C4F790199CFC8
:1007A000DF91CF911F910F91FF90EF90DF90CF904D
:1007B000BF90AF909F908F907F906F90089580EA48
:1007C00080930E0314D173D346D280E190E022D1FE
:1007D00080930D0380E890E01DD180930C03AFE877
:1007E000B3E0EFE0F3E02FE933E08AE01D9280838D
:1007F00081838283838384838583868387833896FA
:100800002A173B0799F708958F9381E08093A003FF
:100810008F9118958091A0031092A00308958823CA
:1008200011F05D9808955D9A0895882311F05E98FF
:1008300008955E9A0895882311F05F9808955F9A4D
:1008400008950895882319F02D9A259A08952D98D2
:10085000FCCF882319F025982D9A08952D98259A74
:100860000895882319F02D9A259A089525982D9892
:100870000895882319F02E9A269A08952E98FCCF71
:10088000882319F026982E9A08952E98269A08956E
:10089000882319F02E9A269A089526982E9808955E
:1008A000882319F02F9A279A08952F98FCCF882330
:1008B00019F027982F9A08952F98279A089588233A
:1008C00019F02F9A279A089527982F9808952C9811
:1008D000249A08952C9A249A089585E38A95F1F72D
:1008E000000008952FEF80E792E021508040904073
:1008F000E1F700C000000895282F392F2115310598
:1009000061F080E090E0EFE9FFE03197F1F700C09F
:100910000000019628173907B1F70895CF93F8948E
:100920001092A00387E0809361001092A00389EFEA
:1009300087BD15BC82E084BD80936E0083E085BDD9
:1009400080919F0380930201CFEFC0930101109229
:100950009F03BDDF559A569A579AC1B9C0930401B7
:1009600017B8C8B97894CF910895282F81E090E006
:10097000A0E0B0E004C0880F991FAA1FBB1F2A95F2
:10098000D2F780959095A095B0958093050125E1CB
:100990002A95F1F70000892F9A2FAB2FBB2782B938
:1009A00085E18A95F1F7000086B1809508959091D0
:1009B0009F038927809302011C9A85E38A95F1F7AA
:1009C00000001C9A0895833059F028F4813039F0E2
:1009D000823021F4FAC3843009F46FC487C3B8C3EA
:1009E00027C4982F81E0953008F080E00895109298
:1009F000A3031092A2031092A1030895882344F048
:100A000091E02091A10382170CF090E0892F0895C6
:100A100080E00895282F392F8091A103843034F588
:100A20006091A2037091A30340E950E0461B570B6D
:100A300042175307ECF091E0980F9093A10397E0D1
:100A40008902F0011124EC55FC4F33832283AB0162
:100A500040545C4F51834083148215821682260FC6
:100A6000371F3093A3032093A20308958FEF0895B7
:100A70008FEF0895CF93DF93C82FD62FBFDF882342
:100A800049F18C2F0C2E000C990B27E0C202F001CB
:100A90001124EC55FC4F268162817381422F50E076
:100AA00046175707BCF4FC01EE0FFF1FEE0FFF1FA8
:100AB000EE0FFF1FE81BF90BEC55FC4F848190E013
:100AC000A081B181A80FB91FDC93019644D484831F
:100AD0002F5F2683DF91CF910895CF93C82F8EDFAC
:100AE00030EA882339F18C2F0C2E000C990B27E06B
:100AF000C202F0011124EC55FC4F268130EA22237A
:100B0000C9F0FC01EE0FFF1FEE0FFF1FEE0FFF1FDE
:100B1000E81BF90BEC55FC4F858190E0A081B18179
:100B2000A80FB91F3C9101966281738114D485830B
:100B300021502683832FCF91089508959FEF980F1A
:100B40009E3050F4E82FF0E0EE0FFF1FE05BFB4F0C
:100B50000190F081E02D099508959FEF980F9E3048
:100B600048F4E82FF0E0EE0FFF1FE05BFB4F8081C1
:100B7000918108958DE995E008959FEF980F9E303B
:100B800040F4E82FF0E0EE0FFF1FE05BFB4F6083C7
:100B900071830895E0E5F4E02EE634E08DE995E018
:100BA00081939193E217F307D9F7E0E5F4E085EB41
:100BB00094E09383828387ED94E095838483089502
:100BC000643080F4413170F4293060F4E62FF0E0B5
:100BD000EE0FFF1FEE0FFF1FE159FB4F8083918344
:100BE000428323830895A7D0E82FF0E0EE0FFF1F84
:100BF000EE0FFF1FE159FB4F828108959CD0E82F33
:100C0000F0E0EE0FFF1FEE0FFF1FE159FB4F838156
:100C10000895CF93DF93D82FE4DE811103C0DF91D5
:100C2000CF910895D0936E0479DEC0E020E040E0DB
:100C30006C2F80E090E0C4DFCF5FC430B9F731D2D1
:100C4000A9DF8D2FC0DEEBCF90916E04981301C009
:100C50000895DFDFFDCF80E0DCCF80916E048E7FD2
:100C6000F3CF80916E048160EFCF80916E048D7F11
:100C7000EBCF80916E048260E7CF80916E048B7F12
:100C8000E3CF80916E048460DFCF80916E04877F14
:100C9000DBCF80916E048860D7CF982F20916E04AF
:100CA00030E0F901EE0FFF1FEE0FFF1FE159FB4F80
:100CB00083818823C1F022812223A1F0E42FF0E078
:100CC000EE0FFF1FEE0FFF1FE159FB4F70E0899FF2
:100CD000600D711D11240190F081E02DE60FF71FCA
:100CE00084910895822F08958093810461E081FFAB
:100CF00062E08BE074C181E0F7CF80918104826073
:100D0000F3CF8091810492E08927EECF9091800407
:100D100081E089278093800461E0913009F462E0EA
:100D20008AE05DC181E080937F04089580E0DCCF9C
:100D300010927F040895E1E080918104811101C047
:100D4000E0E0809180048111E26080917F04811154
:100D5000E460F0E0EE5BFD4F808108951F93CF9338
:100D6000DF93162FC82FD0E0CC0FDD1FCC0FDD1F77
:100D7000C050DE4FE881F981862F09951A83DF91F3
:100D8000CF911F910895CF93DF93C82FD0E0CC0F60
:100D9000DD1FCC0FDD1FC050DE4FE881F98181E0FF
:100DA000099581E08A83DF91CF910895CF93DF93F6
:100DB000C82FD0E0CC0FDD1FCC0FDD1FC050DE4FA1
:100DC000E881F98180E009951A82DF91CF91089539
:100DD000E82FF0E0EE0FFF1FEE0FFF1FE050FE4F79
:100DE00061E09281911160E0B9CF282F90910302C8
:100DF0009923B9F0981779F0E92FF0E0892FEE0FD9
:100E0000FF1FEE0FFF1FE050FE4F9381992359F013
:100E10002913F2CF0895882311F080E008958DE022
:100E200008958DE008958DE00895E82FF0E0EE0F2D
:100E3000FF1FEE0FFF1FE050FE4F838108951F93A9
:100E4000CF93DF93C82FD62F142FCFDF9FEF9C0FA8
:100E50009C30C8F48D30E1F0EC2FF0E0EE0FFF1F76
:100E6000EE0FFF1FE050FE4F9381A82FB0E0AA0FB6
:100E7000BB1FAA0FBB1FA050BE4F13969C93D383DA
:100E8000128381E001C080E0DF91CF911F9108952E
:100E900080E0FACFE2E0F2E080E091E090838F5FC3
:100EA000818334968D30D1F71092330208958DE00E
:100EB00092E09093850480938404909387048093B8
:100EC000860490938304809382040895809186041D
:100ED00090918704909383048093820408951092E4
:100EE0008504109284048091860490918704823452
:100EF000910541F0109287041092860410928304A9
:100F00001092820408958DE092E09093850480937E
:100F1000840480918604909187048234910551F075
:100F20008DE092E0909387048093860490938304ED
:100F30008093820408958091820490918304833485
:100F4000910530F48091860490918704892B51F4A7
:100F500082E490E0909387048093860490938304C6
:100F600080938204089580918404909185049093E5
:100F70008704809386049093830480938204089569
:100F80008091820490918304009799F09C012150F4
:100F90003109019731F0309383042093820480E07B
:100FA000089582E490E0909383048093820481E02A
:100FB000089580E008950F931F93CF93082F192F62
:100FC000C62F662341F08C2FF80109958C2F2DDF59
:100FD000C82F8111F8CFCF911F910F910895CF9312
:100FE000E82FF0E0EE0FFF1FE857FB4FC0816330A2
:100FF000F1F048F0643081F06530B9F46C2F88EE80
:1010000096E0D9DF12C06130E1F0623071F46C2FEC
:1010100086ED96E0D0DF09C06C2F88EE96E0CBDF3E
:1010200061DC6C2F88EE96E0C6DFCF9108956C2FBF
:1010300088EE96E0C0DF51DC6C2F88EE96E0BBDFD7
:10104000F4CF6C2F83EC96E0B6DFEFCFE82FF0E023
:10105000EE0FFF1FE857FB4F6181C1CF0F931F9326
:10106000CF93DF93162F042F9FEF980F9B3028F01C
:10107000DF91CF911F910F910895C82FD0E0FE010D
:10108000EE0FFF1FE857FB4F422F6081812FD7DE05
:10109000882371F3CC0FDD1FC857DB4F18830983FA
:1010A000E7CFF8DEE8E8F4E080EA94E0118210820D
:1010B0003296E817F907D1F70895CF93DF93CDB7AC
:1010C000DEB7AE014B5F5F4FFA0161917191AF01E5
:1010D00084E392E06DD1DF91CF9108958AE492E0AC
:1010E0009F938F93EADF0F900F90089588E2B0DA14
:1010F00060E080E057D062E081E054D061E082E0BF
:1011000051D063E083E04ED06EE678E08DE035DDCF
:1011100062E479E08CE031DD21E040E06AE087E0E4
:101120009DDF20E040E06CE08AE098DF21E043E0D2
:1011300068E081E093DF20E044E063E082E08ECF6E
:101140008AE492E09F938F93B8DF0F900F900895F9
:1011500088E27EDA60E081E025D062E081E022D0A2
:1011600061E082E01FD063E083E01CD060EA78E0B9
:101170008DE003DD62E479E08CE0FFDC21E040E01B
:101180006AE087E06BDF20E040E06CE087E066DF4C
:1011900021E043E068E081E061DF20E044E063E0DB
:1011A00082E05CCFE82FF0E0EE0FFF1FE35AFD4F27
:1011B00028E049E08081918103CD85E692E09F930C
:1011C0008F937BDF0F900F90089588E241DA60E003
:1011D00080E060D062E081E05DD061E082E05AD0E2
:1011E00063E084E057D062E479E086E0C6DC6DED30
:1011F00078E08DE0C2DC20E040E06AE08AE02EDFAB
:1012000020E040E06CE088E029DF21E043E068E096
:1012100081E024DF20E044E063E082E01FDF76CD60
:1012200082E892E09F938F9348DF0F900F9008958C
:1012300088E20EDA60E081E02DD062E081E02AD021
:1012400061E083E027D063E084E024D062E479E0C9
:101250008CE093DC60E179E08DE08FDC20E040E021
:101260006AE087E0FBDE20E040E06CE088E0F6DE4C
:1012700021E043E068E081E0F1DE20E044E063E06B
:1012800082E0ECCE89E992E09F938F9316DF0F9076
:101290000F900895E82FF0E0EE0FFF1FE051FD4F93
:1012A00028E049E0808191818BCC8AEF92E09F9386
:1012B0008F9303DF0F900F90089528E04DE060E0DA
:1012C00084EA94E07DDC28E04DE062E08CE394E089
:1012D00077DC28E04DE061E084ED93E071DC28E00C
:1012E0004DE063E08CE693E06BDC88E2B1D920E06E
:1012F00040E06AE08AE0B2DE20E040E06CE08BE0B3
:10130000ADDE21E045E061E083E0A8DE20E045E0DD
:101310006BE083E0A3DE21E043E068E081E09EDE55
:1013200021E044E064E082E099DEF0DCD3DA65E5B8
:1013300079E08DE022CC43DA01C09CD96BDA8823B6
:10134000E9F372D9C82F803AC0F782E006DCFC01CD
:101350008C2F0995F2CF97FB072E16F4009406D038
:1013600077FD08D011D007FC05D03EF4909581950B
:101370009F4F0895709561957F4F0895EE0FFF1F61
:101380000590F491E02D0994AA1BBB1B51E107C005
:10139000AA1FBB1FA617B70710F0A61BB70B881F05
:1013A000991F5A95A9F780959095BC01CD01089594
:1013B000AFE0B0E0EDEDF9E094C26C017B018A0191
:1013C000DC0117961C921E92169713968C9181FF42
:1013D000DEC12AE0522EF6019381F70193FD85913B
:1013E00093FF81917F01882309F471C0853239F41C
:1013F00093FD859193FF81917F01853221F4B601A0
:1014000090E0DED1E8CF912C612C712CFFE1F71533
:1014100008F445C08B32C1F1F0F48032B9F1833267
:1014200009F43AC0833609F487C0833709F490C0C1
:10143000833509F0B0C0F801A190B1908F01692DFA
:1014400070E076FC02C06FEF7FEFC501A3D14C01C5
:10145000689477F85EC08D32E1F0803351F020ED72
:10146000280F2A3048F18E3209F038C0689476F897
:1014700002C0689470F8F70193FD859193FF819104
:101480007F018111C3CF32C0689471F8689472F8FB
:10149000F2CF689473F8EFCF689474F8ECCF77FCD0
:1014A00025C020ED280F2A3070F476FE05C0959CEB
:1014B000200D1124922EDFCF659C200D1124622E69
:1014C000689475F8D8CF8E3249F476FECFCFD60126
:1014D00016968D919C912F96EFE01FC28C3619F4D1
:1014E000689477F8C8CF883609F4C5CF982F9F7DC8
:1014F0009554933008F096CF0C5F1F4F8FE389838C
:1015000088248394912CAE014F5F5F4F5A01E89479
:1015100077F873FC05C0862D90E08816990630F1A7
:101520008114910449F5662009F455CFB60180E293
:1015300090E046D16A94F7CFD8018C9189830E5FF1
:101540001F4F88248394912CFE0131965F01DFCFD9
:10155000D801AD90BD908D01692D70E076FC02C080
:101560006FEF7FEFC50121D14C01D1CFB60180E2F1
:1015700090E026D16A94CFCFF50177FC859177FE74
:1015800081915F01B60190E01BD161106A94F1E096
:101590008F1A9108C5CF843619F0893609F07DC0BD
:1015A000F80177FE73C061917191819191918F01E2
:1015B000272D2F76822E97FF09C0909580957095E4
:1015C00061957F4F8F4F9F4F689487F82AE030E0F6
:1015D000AE014F5F5F4F5A0123D18A19A82EBA2C52
:1015E000782C86FE0CC0E89470F8A91440F484FEB0
:1015F00005C082FC03C0782D7E7E772EB92C74FE48
:10160000A1C0FE01EA0DF11D8081803309F093C075
:10161000872D897E782E73FC0EC070FEA1C09A2C97
:10162000B61418F4960C9B18B62C862D8B196B14D7
:1016300008F480E0B80EB61408F094C06B1874FE7D
:1016400093C0B60180E390E0BBD072FE08C088E58D
:1016500090E071FC02C088E790E0B601B1D0A91417
:1016600008F48FC0AA94B12C9FEFA91AB90ADE0121
:1016700011964D01AA0EBB1EF50182915F01B601C4
:1016800090E09ED08A149B04B9F74DCF619171917F
:10169000072E000C880B990B8ACF872CE89484F8CE
:1016A0002AE030E0853769F0572D597F852E803745
:1016B00069F110F5883569F18F3609F008CF28E017
:1016C00030E0F80187FE2DC081919191A191B191F7
:1016D0008C879D87AE87BF878F01BE016F5F7F4F6D
:1016E0005B01AB016C857D858E859F8599D08A19BC
:1016F000A82EE89487F873CF883709F0E8CE84FEE7
:1017000002C0689482F820E130E0DBCF689484F86E
:10171000F6CF74FE03C0652F6660862E20E132E0AE
:10172000D0CF81919191AC0160E070E04C875D87F2
:101730006E877F87D1CF72FC02C0B3946CCFB39415
:10174000B39469CF872D8678882309F464CFF5CFC9
:10175000B60180E290E034D083948614C8F365CF5C
:101760008B2CFBCF612C6BCF872D8678882309F4D7
:1017700076CF8BE271FE80E277FC8DE2B60190E0DD
:101780006DCFB60180E390E01BD09A9468CF8FEFC5
:101790009FEFA1CEFC010590615070400110D8F779
:1017A000809590958E0F9F1F0895FC0161507040A9
:1017B00001900110D8F7809590958E0F9F1F089586
:1017C0000F931F93CF93DF93182F092FEB018B817A
:1017D00081FD09C01FEF0FEF812F902FDF91CF9177
:1017E0001F910F91089582FF14C02E813F818C813B
:1017F0009D81281739073CF4E881F981CF010196D2
:101800009983888310838E819F8101969F838E8325
:10181000E3CFE885F985812F0995892BA1F3DACFEC
:10182000FA01AA27283051F1203181F1E8946F9311
:101830006E7F6E5F7F4F8F4F9F4FAF4FB1E03ED0B7
:10184000B4E03CD0670F781F891F9A1FA11D680F55
:10185000791F8A1F911DA11D6A0F711D811D911D88
:10186000A11D20D009F468943F912AE0269F1124FD
:101870003019305D3193DEF6CF010895462F477061
:10188000405D4193B3E00FD0C9F7F6CF462F4F70BC
:10189000405D4A3318F0495D31FD4052419302D01A
:1018A000A9F7EACFB4E0A6959795879577956795C0
:1018B000BA95C9F700976105710508959B01AC01C0
:1018C0000A2E06945795479537952795BA95C9F7E7
:1018D000620F731F841F951FA01D08952F923F92C2
:1018E0004F925F926F927F928F929F92AF92BF9230
:1018F000CF92DF92EF92FF920F931F93CF93DF93DC
:10190000CDB7DEB7CA1BDB0B0FB6F894DEBF0FBE38
:10191000CDBF09942A88398848885F846E847D8485
:101920008C849B84AA84B984C884DF80EE80FD8087
:101930000C811B81AA81B981CE0FD11D0FB6F894FD
:10194000DEBF0FBECDBFED010895F894FFCFCA02F0
:10195000AC02AD02AE02AF02B002B102CA02B202E4
:10196000B302B402B502B702B602B802BA02BC02B0
:10197000BE02C002C202C402C602C802CA02CC022F
:10198000CE02D002D202D402D602D802DA02DC029F
:10199000E702F002F002F002E802E902F002EA02D5
:0A19A000EB02EC02ED02EF02EE0292
:1019AA002104000022040000290400003104000080
:1019BA0039040000400400004804000050040000FC
:1019CA00570400005F0400000F0400001504000023
:1019DA001B040000000000020000000005030000D4
:1019EA00000000010201030303035B4B65796D618B
:1019FA00703A20636C61737369635D0A00BC012CE1
:101A0A00017401E4005B4B65796D61703A204170A5
:101A1A00706C6520322028752F6C206361736529EC
:101A2A005D005B4B65796D61703A204170706C6541
:101A3A00203220434150535D003130474554412400
:101A4A002830293A413D4153432841242830292945
:101A5A003A41242831293D2243544C2B222B434816
:101A6A0052242841202B203634293A3F2227223B70
:101A7A00412428413C3332293B2227203D20223B66
:101A8A00413A4946413C3E33474F544F31300D00AD
:101A9A0024034C02DC02940204025B4B6579626403
:0A1AAA003A20536F6C2D32305D00BE
:00000001FF
